:020000040800F2
:10000000001000201D0F0008190F0008170F00082E
:1000100000000000000000000000000000000000E0
:10002000000000000000000000000000190F0008A0
:100030000000000000000000190F0008190F000860
:10004000170F0008170F0008170F0008170F0008F8
:10005000170F0008170F0008170F0008170F0008E8
:10006000170F0008170F0008170F0008170F0008D8
:10007000170F0008170F0008170F0008170F0008C8
:10008000170F0008170F0008170F0008170F0008B8
:10009000170F0008C5040008170F0008F104000836
:1000A000170F0008170F0008170F0008E9000008D5
:1000B000170F0008170F0008170F0008170F000888
:1000C00070B50600017800290AD00024054D89B2D8
:1000D000280000F05AFE0134E4B2315D0029F6D167
:1000E00070BDC0460038014010B5184B1B689B0618
:1000F0001ED5174B1B689B061AD5144800F053FEFB
:10010000C0B2144A11784B1CDBB21370124A50541F
:100110000021D1540D2806D1104B1B6810009847C0
:1001200000220C4B1A70094A116880230B4313609C
:10013000064B1B681B0608D5054B1B681B0604D520
:10014000024A136880218B43136010BD00380140C0
:100150001C38014018000020240000201C00002052
:10016000F0B587B005000F00002822D0002600E07F
:1001700026000A21280000F0B5FF303101AB995567
:10018000741CE4B20A21280000F026FF051EEFD1FE
:10019000002C0ED0631E01AA944663443A00A11EAF
:1001A0008E1B664419781170013B0132B342F9D1BC
:1001B00002E030233B70012400233B5507B0F0BD23
:1001C00000B587B001A9FFF7CBFF01A8FFF778FFC3
:1001D00007B000BDF0B5474680B480460024084F04
:1001E000084EE519A05B43465843642100F07EFFAA
:1001F00028800234422CF4D104BC9046F0BDC046A5
:1002000030000020F415000810B5184B984203DDAB
:100210000022174B1A6009E0C3171B1ADB0FC20F2D
:100220009B1A144A12685343114A1360C317C0182B
:100230005840114B1860114B984203D80022104BC4
:100240001A7009E0010C0E4B1970FF23194001319F
:1002500000F0C2FE084B1860074B1A68094B1A6081
:10026000074B1A78084B1A6010BDC046809698005C
:10027000A40000207800002080000020FFFF000084
:10028000C50000202C4401403044014010B5354BDE
:100290001A68354B1B689A4263D0334B1A68314B4E
:1002A00019681B68521AD11752184A409B10D91767
:1002B0005B184B409A4208DA2B4B1B68294A12689C
:1002C0009B1ADA179B18534005E0264B1B689B10BE
:1002D000DA179B185340002B04D1234B1A68214B8B
:1002E0001A603AE01F4A12681F490868C117091AC4
:1002F000C90FC00F081AD117891AC90FD20F8A1A4D
:1003000090420FD1174A1168174A1268914204DAD5
:1003100014490A689B180B601FE012490A68D31A37
:100320000B601AE00F4A11680F4A1268914204DA12
:100330000C490A68D31A0B6003E00A490A689B1843
:100340000B60084B1B68DA179B185340074A93420F
:1003500003DD044A13685B421360024B1868FFF721
:1003600053FF10BDB4000020880000208813000057
:1003700070B5FFF78BFF4C4B1A684C4B1B689A42C9
:100380000BD14B4B1B68002B07D00022484B1A6047
:10039000F0221206454B1A6085E0454A1068424932
:1003A0000B68C3180B601268424B1B68D31803D547
:1003B0008033404A136007E07F2B02DC3D4A136024
:1003C00002E0803B3B4A13603A4B1B685811C1B2B4
:1003D000DA17D20E9B181F2423409B1A2022D21A10
:1003E000D2B2C0072DD53448E03423405B001C5AFC
:1003F0005200155A012911D19026F605300000F05F
:10040000EDFB0221300000F0EBFB0821300000F092
:10041000E7FB1021300000F0E1FB40E09026F605FC
:100420000121300000F0DCFB0221300000F0D6FB9F
:100430000821300000F0D2FB1021300000F0D0FB8A
:100440002DE01D485200145AFF2213405B001D5A34
:10045000002912D19026F6050131300000F0BEFBD4
:100460000221300000F0BCFB0821300000F0B6FB98
:100470001021300000F0B4FB11E09026F6050121B8
:10048000300000F0ADFB0221300000F0A7FB082196
:10049000300000F0A5FB1021300000F09FFB074B5F
:1004A0001D60074B1C6070BD740000200800002018
:1004B000A4000020BC0000203000002034040040D4
:1004C0003804004010B50121074800F0D9FB00288E
:1004D00009D00121044800F0DAFB044B1B68002B13
:1004E00001D0FFF745FF10BD00440140A4000020EB
:1004F00010B5724B1B681A071DD5DB0306D5002209
:100500006F4B1A706F4A704B1A600EE001236C4AF1
:10051000137000216D4A11706D4A6E490A606E4970
:100520000A60664A11680B4313606C4A116808231D
:100530000B431360C0E05A071BD5644B1B78DBB23A
:10054000092B00D9B8E0664800F060FC5F4B1B78CF
:10055000002B02D1634B187005E05C4B1B785C4AA2
:10056000D318013B1870594A13780133DBB213706A
:10057000A2E09A0708D5544A1368591C11601B78E9
:10058000DBB2594A136097E09A0600D48DE05448D4
:1005900000F028FC514A116820230B431360484B9C
:1005A0001B78002B00D187E04E4B1B78DBB2442B2D
:1005B00000D981E09B004D4AD3589F464C4B1A68A6
:1005C000404B1A6078E0434B1B681A68484B1A602E
:1005D00072E0404B1B681A68464B1A606CE0454B52
:1005E0001A68384B1A6067E03A4B1B681868424B30
:1005F0001860FFF709FE5FE0364B1B681B68DA17CF
:100600009B1853403D4A136056E0324B1B681968F3
:100610003B4C21608020C00500F046FB2168394832
:1006200000F0DAFC384B186046E02A4B1B6818686B
:10063000FFF7D0FD40E0284B1B681C68334B1C6063
:10064000314B186800F07AFF211C00F03BFE00F0EF
:1006500053FF294B18602E4A10601868FFF7D4FD2D
:100660002AE01D4B1B681C682A4B1C60264B18682F
:1006700000F064FF211C00F025FE00F03DFF244B3C
:10068000186019E0224B1A680E4B1A6014E01A4BDE
:100690001A680C4B1A600FE01F4B1A68094B1A605E
:1006A0000AE001221D4B1A7006E0DB0604D50B4A56
:1006B000116810230B43136010BDC046185400404E
:1006C0009D000020940000207C0000209C00002061
:1006D000A8000020C0000020840000201C5400401E
:1006E00000540040C4000020285400403816000880
:1006F0007400002008000020B400002078000020D2
:100700000C000020006CDC02040000209800002097
:1007100088000020A0000020A4000020200000206D
:10072000F0B557464E464546E0B43C20FFF752FD33
:1007300000F022FA904800F0BBFA904800F0B8FAB6
:100740008F4800F0B5FA8F4800F0B2FA9025ED0519
:100750001F2300220121280000F045FA8A4B0022C5
:100760000221280000F03FFA04220121280000F0B5
:1007700057FAC0220121280000F052FA834C96213A
:100780008901200000F0C4FA0821200000F0CCFA12
:100790000021200000F0DEFA0021200000F0D2FA53
:1007A0000821200000F0DEFA0021200000F0E0FA2D
:1007B000200000F0E5FA764800F07AFA172000F001
:1007C000F5FB744C200000F0C9F9C026F600330098
:1007D00000220221280000F006FA3200042128003D
:1007E00000F01EFA200000F0E7FA200000F0FFFA07
:1007F000200000F00FFB0021200000F013FB082276
:100800000021200000F058FB200000F041FB2000F8
:1008100000F046FB604B1978200000F0EDFA5F4ACB
:100820001368802109020B4313603E21200000F071
:100830003FFB200000F0D6FA594800F039FA1520A5
:1008400000F0B4FB9220FF3000F040FA554B1968DD
:10085000554C200000F028FA544B9946544B4A4618
:100860001A600021200000F021FA200000F012FAA6
:10087000200000F014FA0121200000F0FDF94D4A9B
:1008800000241460802189004B4B19604B4B1C6085
:1008900001214B4B19604B4F3B6868208246034354
:1008A0003B60494B18680843186048480460386842
:1008B0008446D020C00180466046464630433860BA
:1008C0001868102707431F60414F3C60414F38684C
:1008D000564606433E60186880277F0138431860FB
:1008E0003D4B1C60106880230343136013680B4367
:1008F00013603A4B1960280000F070F908212800B5
:1009000000F06CF90221280000F06AF9102128009B
:1009100000F066F9324B4A461A60324B1C600023E5
:10092000314A1360314A1360314B9846314F324E91
:1009300043461B78002B14D0304D00242000FFF7D5
:100940003FFC3800FFF7BCFB2888FFF739FC30007C
:10095000FFF7B6FB01340235212CEFD10022244BE6
:100960001A70274B1A88002AE2DD0023C0460133A3
:100970009342FBDBDCE7C0468103000091020000EC
:10098000920200000E030000C4060000003801407F
:10099000950300000054004002000020085400406D
:1009A000110300000C00002000440140FFFF000084
:1009B0002C440140000400402C0400402804004066
:1009C0001404004018040040200400403404004097
:1009D000380400401C04004040040040780000201F
:1009E00080000020A4000020A0000020980000202B
:1009F00020000020501700084C170008300000208D
:100A00000000002000B5002306281AD8012200F0BB
:100A1000D9FA06080A0E141204000B4B04E00A4B24
:100A20000CE00A4B0AE0094B1B685B0C08E0074B23
:100A30001B685B0E04E0064B00E0064B1B685B087E
:100A40001340180000BDC0463410024000100240A0
:100A5000201002402410024010B504002000FFF7CF
:100A6000D1FF0028FAD010BD00B506281CD800F030
:100A7000A9FA06080A15110F04000C4A04E00B4AF3
:100A800009E00B4A07E00A4A80211368490209E09D
:100A9000084A00E0084A1368012103E08021044A63
:100AA000490413680B43136000BDC0463410024074
:100AB000001002402010024024100240013800B50E
:100AC00005281AD800F07EFA03080E19191403211C
:100AD0000A4A13688B430FE00321084A13688B43CB
:100AE000023908E00321054A13688B43013902E00B
:100AF0000321024A13680B43136000BD0410024037
:100B0000034A044B11680B40184310607047C046FD
:100B100004100240FFFFC3FF034A044B11680004A6
:100B20000B4018431060704704100240FFFFFEFFA7
:100B3000034A044B11680B40184310607047C046CD
:100B400004100240FFF8FFFFF021034A13688B43B3
:100B5000184310607047C04604100240044B98428E
:100B600004D11021034A13688B4313607047C046B9
:100B7000005400403010024010B50120FFF774FF10
:100B80000120FFF769FF0120FFF798FF0020FFF722
:100B9000DBFF0020FFF7CCFF00F0A8F8012000F0F9
:100BA000ADF8A0208003FFF7ABFF0020FFF7B4FFF4
:100BB0000320FFF759FF0320FFF74EFF0320FFF745
:100BC0007DFF034B034A1360034A136010BDC04608
:100BD000006CDC02140000201000002081617047CE
:100BE000090481617047F7B5002500910468C16868
:100BF0000193019E01232E411E420BD003266F005C
:100C0000BE40F643344031401600009BBE40BB401E
:100C100031431C430135102DEBD10460C160F7BD99
:100C2000F7B500250F27046A436A0192019E01224D
:100C30002E41164206D03A00AE00B24094430A005C
:100C4000B24014430135082DF0D100250F272E00A6
:100C5000019A0836324116000122164206D03A00A7
:100C6000AE00B24093430A00B24013430135082D51
:100C7000EDD104624362F7BDC3681943C160704798
:100C8000036919400800411E8841C0B27047C9433A
:100C90000161704702220368934303607047012299
:100CA00003681343036070478162704701637047B4
:100CB000054A43099B181F2210401E3A82401968BA
:100CC0000A431A607047C04600100240064A4309B2
:100CD0009B181F2210401E3A824019681143196068
:100CE0001968914319607047001002401021024AB0
:100CF00013680B4313607047002002400721034A2A
:100D000013688B43184310607047C04600200240B0
:100D1000044B10B51B6804004808C01800F05CF9CB
:100D2000E06010BD14000020082903D10268044BC4
:100D3000134003E0802203685201134303607047AD
:100D4000FFEFFFFF4268024B1340194341607047B9
:100D5000FFCFFFFF0268024B134019430160704749
:100D6000FFF9FFFF0C2203689343194301607047AA
:100D70008268024B1340194381607047FFFCFFFFFC
:100D80000122036813430360704770B50D0004002F
:100D900000F00DF82900200000F001F870BDC90531
:100DA000C90D81627047406AC005C00D704780233D
:100DB000C2691A42FCD07047064B10B5984204D065
:100DC000054B984204D1054800E00548FFF77EFF37
:100DD00010BDC046005400400058004016020000FC
:100DE00015020000012203681343036070470122CB
:100DF0000368934303607047490081608268024B37
:100E0000134083607047C046FFFBFFFF406AC0B2DB
:100E1000704700000268024B134003607047C046F1
:100E2000FFEFFFFF0268034B090213401943016003
:100E30007047C046FFF0FFFF036909071B011B094C
:100E400019430161704700000269034B0905134013
:100E5000194301617047C046FFFF0FFF0269034B52
:100E600009041340194301617047C046FFFFF0FFBA
:100E70000269034B09021340194301617047C046E0
:100E8000FF00FFFFFF22036993431943016170478D
:100E90000268024B134003607047C046FFFFFDFF2E
:100EA0004268024B134043607047C046FFF7FFFFA4
:100EB000036819430160704710B50400012914D07C
:100EC000022927D09208013AD1B2FFF7B5FF1321CA
:100ED0002000FFF7D7FF0F212000FFF7C9FF0221F5
:100EE0002000FFF7BBFF042111E0D208013AD1B284
:100EF000FFF7A2FF09212000FFF7C4FF0321200014
:100F0000FFF7B6FF03212000FFF7A8FF0321200011
:100F1000FFF79AFF10BDFEE770470000002270B592
:100F20001748184D1849131854198B4203D22468D6
:100F300004321C60F7E70021144A934202D2196080
:100F40000433FAE78021124A89001368114C0B43DD
:100F50001360114B9C4202D208CC9847F9E70F4C22
:100F60000F4B9C4202D208CC9847F9E7FFF7D8FB19
:100F70000C4C0D4B9C4202D208CC9847F9E770BD4F
:100F800000000020D417000818000020C80000202E
:100F900014ED00E0D4170008D4170008D417000897
:100FA000D4170008D4170008D41700084309044ACE
:100FB0009B009B181F2210401E3A82401A60704707
:100FC00000E100E002B4714649084900095C4900AB
:100FD0008E4402BC7047C046002243088B4274D343
:100FE00003098B425FD3030A8B4244D3030B8B422A
:100FF00028D3030C8B420DD3FF22090212BA030C33
:101000008B4202D31212090265D0030B8B4219D313
:1010100000E0090AC30B8B4201D3CB03C01A524133
:10102000830B8B4201D38B03C01A5241430B8B427B
:1010300001D34B03C01A5241030B8B4201D30B0364
:10104000C01A5241C30A8B4201D3CB02C01A52418B
:10105000830A8B4201D38B02C01A5241430A8B424E
:1010600001D34B02C01A5241030A8B4201D30B0237
:10107000C01A5241CDD2C3098B4201D3CB01C01A51
:10108000524183098B4201D38B01C01A524143095B
:101090008B4201D34B01C01A524103098B4201D349
:1010A0000B01C01A5241C3088B4201D3CB00C01AB6
:1010B000524183088B4201D38B00C01A524143082E
:1010C0008B4201D34B00C01A5241411A00D2014653
:1010D000524110467047FFE701B5002000F0F0F8DC
:1010E00002BDC0460029F7D076E7704703460B43A0
:1010F0007FD4002243088B4274D303098B425FD311
:10110000030A8B4244D3030B8B4228D3030C8B423C
:101110000DD3FF22090212BA030C8B4202D3121222
:10112000090265D0030B8B4219D300E0090AC30BF7
:101130008B4201D3CB03C01A5241830B8B4201D3A4
:101140008B03C01A5241430B8B4201D34B03C01A8D
:101150005241030B8B4201D30B03C01A5241C30A05
:101160008B4201D3CB02C01A5241830A8B4201D376
:101170008B02C01A5241430A8B4201D34B02C01A60
:101180005241030A8B4201D30B02C01A5241CDD205
:10119000C3098B4201D3CB01C01A524183098B4250
:1011A00001D38B01C01A524143098B4201D34B0139
:1011B000C01A524103098B4201D30B01C01A52419C
:1011C000C3088B4201D3CB00C01A524183088B4223
:1011D00001D38B00C01A524143088B4201D34B000C
:1011E000C01A5241411A00D201465241104670477E
:1011F0005DE0CA0F00D04942031000D34042534083
:1012000000229C4603098B422DD3030A8B4212D342
:10121000FC22890112BA030A8B420CD38901921174
:101220008B4208D3890192118B4204D389013AD0B1
:10123000921100E08909C3098B4201D3CB01C01A86
:10124000524183098B4201D38B01C01A5241430999
:101250008B4201D34B01C01A524103098B4201D387
:101260000B01C01A5241C3088B4201D3CB00C01AF4
:10127000524183088B4201D38B00C01A5241D9D20C
:1012800043088B4201D34B00C01A5241411A00D28D
:101290000146634652415B10104601D34042002B89
:1012A00000D54942704763465B1000D3404201B508
:1012B000002000F005F802BD0029F8D016E77047BD
:1012C0007047C046F0B5564644465F464D46F0B4BA
:1012D00044024600C70F83B08846650A360EBA46F8
:1012E0003DD0FF2E22D00023EC00802599469B465E
:1012F000ED0425437F3E43465C025800DB0F640A41
:10130000000E984636D0FF2830D080230021E4001C
:10131000DB041C437F38301A01904846424608439C
:10132000724E800030587A4013008746002D44D119
:1013300008239946063B9B46DDE70122FF20002457
:101340001A406402C305640AD2071C4314432000F8
:1013500003B03CBC90469946A246AB46F0BD002D7A
:1013600020D104239946033B9B46C4E7002C17D1A8
:10137000022102E0002C0AD10121321A01924A46D0
:1013800043460A435A48920082587B4097462000C1
:1013900000F012F9431F76309C4040420021BAE72A
:1013A0000321B8E7280000F007F9431F9D40002300
:1013B0007630464299469B469DE70C239946093B69
:1013C0009B4698E780240022E403FF20B9E700242D
:1013D000C2468B465A465346022AAED0032A7DD0D7
:1013E000012A31D1012200201A400024A9E701225C
:1013F000101A1B2856DD1A4000200024A1E7802384
:10140000DB031D424BD18023DB032B435C02640AC8
:101410003A00FF2095E76D016001854230D2019AC4
:101420000024013A01921B220127290064006D006B
:10143000002901DBA84201D82D1A3C43013A002AB9
:10144000F3D16A1E95412C4301987F300028CEDDF0
:10145000620704D00F222240042A00D00434220163
:1014600003D5244A019814408030FE2800DD64E74B
:101470000122A401640AC0B21A4062E72C00A9E765
:101480002D1A1A220124CFE76B02BCD50024802339
:10149000DB031C436402640A4246FF2051E71C42FE
:1014A000B3D1F4E721002022C140101A8440621E0B
:1014B00094410C43620704D00F222240042A00D03A
:1014C0000434620104D5012201201A40002438E7C7
:1014D0000122A401640A1A40002032E78023DB03C2
:1014E0001C436402640A5246FF202AE7541700088E
:1014F00094170008FFFFFFF74302590A4300C20F89
:101500001B0E00207E2B0EDD9D2B0DDC80200004A9
:101510000143952B0BDC9620C31AD9400B0058428F
:10152000002A00D118007047034BD018FBE7963B08
:1015300099400B00F3E7C046FFFFFF7F70B5041E24
:1015400028D000F039F89E231B1A962B0ADC96222D
:10155000D21A94406202520AD8B25202520AC0050C
:10156000104370BD992B18DC9922D21A9440114A6D
:101570002240610704D00F210C40042C00D004321B
:10158000510103D50B4B1A409F231B1A9201520A9B
:10159000D8B2E2E700200022DFE705222500121A78
:1015A000B921D5402200C91A8A40541EA2412C00FC
:1015B0001443DCE7FFFFFFFB1C2101231B049842BF
:1015C00001D3000C10391B0A984201D3000A0839D4
:1015D0001B09984201D30009043902A2105C40188B
:1015E0007047C0460403020201010101000000002F
:1015F000000000000000320064009600C800F900FE
:10160000290159018801B601E3010E023902620283
:101610008A02B002D402F7021803360353036E03A2
:1016200087039E03B203C403D403E103EC03F50371
:10163000FB03FF0300040000B8060008B80600081A
:10164000BC050008C6050008D2050008DE05000834
:10165000E8050008F80500080A0600082A06000840
:101660003606000862060008840600088E06000898
:1016700098060008B8060008B8060008B806000872
:10168000B8060008B8060008B8060008B806000842
:10169000B8060008B8060008B8060008B806000832
:1016A000B8060008B8060008B8060008B806000822
:1016B000B8060008B8060008B8060008B806000812
:1016C000B8060008B8060008B8060008B806000802
:1016D000B8060008B8060008B8060008B8060008F2
:1016E000B8060008B8060008B8060008B8060008E2
:1016F000B8060008B8060008B8060008B8060008D2
:10170000B8060008B8060008B8060008B8060008C1
:10171000B8060008B8060008B8060008B8060008B1
:10172000B8060008B8060008B8060008B8060008A1
:10173000B8060008B8060008B8060008B806000891
:10174000B8060008B8060008A20600080D0A000046
:101750002D000000161400083A130008F8130008C2
:10176000D0130008F8130008C4130008F813000889
:10177000D01300083A1300083A130008C4130008F5
:10178000D01300087C1400087C1400087C140008A6
:10179000FE1300083A1300083A130008E413000887
:1017A000CE130008E4130008C4130008E413000873
:1017B000CE1300083A1300083A130008C4130008B7
:1017C000CE1300087C1400087C1400087C14000868
:0417D0008814000871
:1017D4003200340080BB0000FFFFFF00E80300007C
:0817E40000127A0000127A00E5
:0400000508000F1DC3
:00000001FF
